:10000000F9C0000013C1000011C100000FC10000C1
:100010000DC100000BC1000009C1000007C10000B4
:1000200005C1000003C1000001C100000C94BC1117
:10003000FDC00000FBC00000F9C000002BC700009D
:10004000F5C00000F3C00000F1C0000084C1000052
:10005000EDC00000EBC00000E9C00000E7C00000F8
:10006000E5C00000E3C00000E1C00000DFC0000008
:10007000DDC0000018034100560052004900530043
:10008000500020006D006B004900490000000C0387
:10009000410054004D0045004C00000004030904D9
:1000A00012011001FF000010EB0304210002010205
:1000B00003014000410142430309000A000A000B0A
:1000C000000C000D000D000E000F001000100012BB
:1000D0000013001300140016001600180019001A6F
:1000E000001C001D001F0020002200230025002707
:1000F0000029002B002E0030003200340037003A77
:10010000003D004000430046004A004E00520055AA
:10011000005A005E00630068006D00730078007E86
:100120000084008B0091009900A000A900B100B9E3
:1001300000C300CC00D600E100EC00F70004011180
:10014000011E012D013B014B015B016C017D019101
:1001500001A501BA01CF01E601FE01160231024CF0
:10016000026A028802A802CA02ED02110338036083
:10017000038B03B803E70318044B048104B904F5A7
:100180000434057505B90501064E069D06EF0648BF
:1001900007A30704086508D0084009B6092B0AAB75
:1001A0000A300BC30B510CEE0C8F0D400EF60EAF48
:1001B0000F681047111412F512ED13E214F015F93F
:1001C000161B185C19911AE51B251D831E0320AB15
:1001D00021302332250F27F128F82A1A2D492FA183
:1001E000311434A1364539173C1A3F34426045DF9B
:1001F00048704C0011241FBECFEFD2E0DEBFCDBF50
:1002000011E0A0E0B1E0E0E4F7E202C005900D9259
:10021000A23AB107D9F711E0A2EAB1E001C01D92FC
:10022000A53BB107E1F744D00C949E13E9CE95B1FC
:100230009F71982B95B9089584B7877F84BF88E113
:100240000FB6F89480936000109260000FBE90E0AB
:1002500080E80FB6F89480936100909361000FBE20
:1002600084B1806E84B985B18F7185B90C94AD115C
:1002700080ECDDCF80E4DBCF82E060E842E30E94E7
:100280001411882311F080E801C080E4D0CF8EB330
:10029000843069F4C3D182E08093E9008091E80062
:1002A00082FF05C080ECC3DF73D080E8C0CF089523
:1002B000C3DF66D080E4BBDF7894489B02C090E047
:1002C00001C090E285B18F7D892B85B9E0DF0E9466
:1002D0006913F3CF01C00895F9011082923029F01B
:1002E000933049F0913071F528C0908380E290E01E
:1002F000EEE1F1E02BC0813051F0813028F0823006
:1003000049F08330F9F40BC0ECE9F0E005C0EEE809
:10031000F0E002C0E4E7F0E0849190E017C0809143
:10032000000190E022E330E030930F0120930E01B2
:1003300022E02083E0E0F1E009C082E190E0E0EA21
:10034000F0E004C080E090E0E0E0F0E0DA01119637
:10035000FC93EE93089578941F920F920FB60F922C
:1003600011248F938AB5882321F08AB581508ABDE4
:1003700001C015BC8F910F900FBE0F901F90189564
:100380008BE987BD82E084BD80936E002CD1B0C51F
:100390000F931F93CF93DF930F92CDB7DEB71091DA
:1003A000F10084E68ABD85E085BD143109F4CAC038
:1003B000153110F51A3009F4ACC01B3068F4143054
:1003C00038F4123008F054C0113009F0D3C033C0F3
:1003D000163009F0CFC077C0113109F4AEC0123128
:1003E00020F4103109F0C6C0A6C0123109F4ADC026
:1003F000133109F0BFC0A3C0193109F4ABC01A31E1
:1004000068F4163109F49EC0163108F498C017310B
:1004100009F4A0C0183109F0ADC099C01D3109F42C
:100420009CC01D3108F493C0103509F49AC01135F1
:1004300009F0A0C094C08091E8008B778093E80019
:1004400082E08093E9008091EC0081608093EC0071
:100450001093F1001092F1008AE08093F1008EE396
:1004600091E06AE070E040E050E00E94E90E98C040
:100470000091F100123011F46091F1008091E800D8
:100480008B778093E80082E08093E9008091EC0014
:1004900081608093EC001093F100802F6983BFD0BE
:1004A0006981123039F481FF0CC01092F100802F65
:1004B000C6D076C080FF05C01092F100802FB7D063
:1004C0006DC080EC6BC086EA91E064E070E040E0D3
:1004D00050E00E94890F8091E8008B778093E800BC
:1004E00082E08093E9008091EC0081608093EC00D1
:1004F0008091A6019091A701A091A801B091A901B6
:10050000B7FF03C081E08093A50186E08093F100EE
:100510000FC08091E8008B778093E80082E08093A1
:10052000E9008091EC0081608093EC001093F10071
:100530001092F10035C033D438C0FDD336C0812FBE
:10054000BDD033C0812FE6D130C0ADD32EC0812FB6
:100550007ED22BC0812FD4D228C013D326C0ECD694
:1005600024C01AD722C08091E8008B778093E800DE
:100570000E9447118091F2008034A9F38091E80035
:100580008B778093E80082E08093E9008091EC0013
:1005900081608093EC001093F10089EC8093F1006E
:1005A0008091E8008E778093E80015BC0E94471187
:1005B00082E08093E9008091EC008E7F8093EC00D4
:1005C0000F90DF91CF911F910F9108959AE0E9E488
:1005D000F1E02081821729F033969150D1F7E0E0C5
:1005E000F0E0CF010895CF93DF9380E090E00E9488
:1005F0008413D82F81E090E00E948413C82FDF3F3E
:1006000021F08EE9E3DFFC01D283CF3F21F088E9BE
:10061000DDDFFC01C283DF91CF9108950895D6DF1D
:10062000009719F0FC018181089580E00895CEDFE4
:10063000009719F0FC018281089580E008951F93CE
:10064000CF93DF930F92CDB7DEB7182F6983BEDF4C
:10065000FC016981009761F062831E3919F480E022
:1006600090E004C0183921F481E090E00E948C13DE
:100670000F90DF91CF911F91089590916701992379
:1006800029F08EBD0DB407FEFDCF089599C4909159
:100690006701992331F08EBD0DB407FEFDCF8EB5F5
:1006A00008958EC480916701882331F01EBC0DB47B
:1006B00007FEFDCF8EB5089580E082C44F925F9211
:1006C0006F927F928F929F92AF92BF92CF92DF9262
:1006D000EF92FF920F931F93CF93DF93CDB7DEB7C7
:1006E000C950D1400FB6F894DEBF0FBECDBF182F52
:1006F000CE01019669E070E040E050E00E94390FC1
:100700006A8179817A83698381E06130780788F032
:100710008091E8008B778093E80082E08093E90085
:100720008091EC0081608093EC001093F10080ECEC
:10073000D2C0CE010A9640E050E00E94390F898174
:100740009A810A968F739070009739F48091E8002F
:100750008B778093E8000E9447118091E8008B77A7
:100760008093E80082E08093E9008091EC00816052
:100770008093EC00133111F4D88401C0D9844090E7
:10078000A6015090A7018AE0882E912C8C0E9D1E08
:10079000AA24BB24EE24FF2498E0C92E7724739466
:1007A00063C0F40161904F010B818091A501882302
:1007B00019F059D41092A5018D815FDF8091A701B6
:1007C0005CDF8091A60159DF862D57DF133119F4C4
:1007D0008D818C258D83E114F10479F46D1469F019
:1007E0008F81A0FE04C0133111F4886001C0877F9F
:1007F0008F83E090A601F090A70100FD11C0E114E5
:10080000F10421F403FD02C0097F0260802FB701CB
:100810004D2D2C810F8130D4882369F5EE24FF24DF
:10082000A0FC02C01531E9F48091A6019091A701C6
:10083000A091A801B091A9010196A11DB11D8093BD
:10084000A6019093A701A093A801B093A901133129
:1008500041F4A070B0700097A105B10511F4709239
:10086000A5010894A11CB11C89819A81A816B9061A
:1008700008F497CF80E09B8197FF2BC08E81FDDE2F
:10088000852DFBDE842DF9DE80E0F7DE8B8185FF90
:1008900006C0E114F10419F48F7C80618B838B8195
:1008A000B7014D2D2C810F81E7D3133191F4409185
:1008B000A6015091A7016091A8017091A9016070F3
:1008C0007070411551056105710519F491E090931F
:1008D000A5011093F1008093F1008091E8008E77DC
:1008E0008093E800C75FDE4F0FB6F894DEBF0FBEFF
:1008F000CDBFDF91CF911F910F91FF90EF90DF90CF
:10090000CF90BF90AF909F908F907F906F905F90AF
:100910004F900895DF92EF92FF920F931F93CF9322
:10092000DF9300D00F92CDB7DEB7F82ECE0101963F
:1009300063E070E040E050E00E94390F89819A81C5
:1009400099838A838091E8008B778093E80082E026
:100950008093E9008091EC0081608093EC00F0923C
:10096000F1001092F10000E010E028E0D22EEE2419
:10097000E39448C08091A501882319F074D31092A4
:10098000A5018B817ADE8091A70177DE8091A60197
:1009900074DE88DE8093F1008091E80085FD07C059
:1009A0008091E8008E778093E8000E94471124E14F
:1009B000F21619F48B818D258B8300FD03C086E12F
:1009C000F816F1F48091A6019091A701A091A801D9
:1009D000B091A9010196A11DB11D8093A60190932C
:1009E000A701A093A801B093A90126E1F21641F056
:1009F000A070B0700097A105B10511F4E092A501B7
:100A00000F5F1F4F89819A810817190708F4B2CF29
:100A10001092F1009091E8008091E8008E77809329
:100A2000E80095FD09C00E9447118091E8008E778B
:100A30008093E8000E9447110F900F900F90DF9174
:100A4000CF911F910F91FF90EF90DF900895CF927B
:100A5000DF92EF92FF920F931F93CF93DF93CDB767
:100A6000DEB729970FB6F894DEBF0FBECDBFD82EE4
:100A7000CE01059665E070E040E050E00E94390F3D
:100A80008091E8008B778093E80082E08093E90012
:100A90008091EC0081608093EC008E010A5F1F4F13
:100AA0007E010894E11CF11C34E0C32EF801819111
:100AB0008F01EDDDF70181937F01CA94B9F7D092E0
:100AC000F1001092F1008D81FE01E80FF11D80818F
:100AD0008093F1001092F1008091E8008E7780936E
:100AE000E80029960FB6F894DEBF0FBECDBFDF91A8
:100AF000CF911F910F91FF90EF90DF90CF900895CD
:100B0000EF92FF920F931F93CF93DF9300D000D00B
:100B1000CDB7DEB7F82ECE01019664E070E040E07C
:100B200050E00E94390F8091E8008B778093E800B5
:100B300082E08093E9008091EC0081608093EC007A
:100B40008E010F5F1F4FE4E0EE2EF80181918F01BF
:100B500094DDEA94D1F7F092F1001092F100109236
:100B6000F1008091E8008E778093E8000F900F905D
:100B70000F900F90DF91CF911F910F91FF90EF9009
:100B80000895FF920F931F93CF93DF93CDB7DEB7F6
:100B9000C250D1400FB6F894DEBF0FBECDBFCE011C
:100BA000019663E070E040E050E00E94390F8E0152
:100BB0000C5F1F4F6981C80170E040E050E00E9467
:100BC000390F8091E8008B778093E80082E0809372
:100BD000E9008091EC0081608093EC008DE18093CE
:100BE000F1001092F100FF240BC08981F81628F45F
:100BF000F801EF0DF11D808101C080E03EDDF3942E
:100C00008B81F81690F300E01CC08981F81650F42F
:100C1000E4E0F0E0EC0FFD1FEF0DF11DF394808197
:100C200036DD01C03FDD8093F1008091E80085FD55
:100C300007C08091E8008E778093E8000E944711FA
:100C40000F5F8A81081708F31092F1009091E80075
:100C50008091E8008E778093E80095FD09C00E949E
:100C600047118091E8008E778093E8000E94471139
:100C7000CE5FDE4F0FB6F894DEBF0FBECDBFDF9163
:100C8000CF911F910F91FF90089506C0EFE9FFE00B
:100C90003197F1F700C00000882321F09AB5815008
:100CA0009923A1F70895FF920F931F93CF93DF939A
:100CB00000D000D000D0CDB7DEB7CE01019666E0FF
:100CC00070E040E050E00E94390F8091E8008B779F
:100CD0008093E80082E08093E9008091EC008160DD
:100CE0008093EC008E010D5F1F4FF4E0FF2EF801A2
:100CF00081918F01C2DCFA94D1F78A81882321F493
:100D00008981C3DF80E001C090D192E19093F1002E
:100D10008093F1008091E8008E778093E80026961A
:100D20000FB6F894DEBF0FBECDBFDF91CF911F91FC
:100D30000F91FF9008950F931F93CF93DF9300D0EF
:100D4000CDB7DEB7CE01019662E070E040E050E042
:100D50000E94390F08EE10E0F80180818B778083C4
:100D600082E08093E900ECEEF0E080818160808396
:100D700089818BDF80E04DD1CFD08A8186DFE1EFA2
:100D8000F0E081E180831082F80180818E7780839A
:100D90000F900F90DF91CF911F910F910895DF92E7
:100DA000EF92FF920F931F93CF93DF93CDB7DEB7F0
:100DB0002F970FB6F894DEBF0FBECDBFCE010596BC
:100DC0006BE070E040E050E00E94390F8091E80055
:100DD0008B778093E80082E08093E9008091EC00BB
:100DE00081608093EC001092A6011092A7011092EE
:100DF000A8011092A9018F8148DFBAD019C0898556
:100E000044DFF80181918F0142DCF70181937F017A
:100E1000DA94A9F78B85882311F1FE01E80FF11D03
:100E200090818A859817D9F080E0F3D08E812DDFEC
:100E300081E0EFD08E8129DF8885982F91509887A7
:100E4000882379F08AB5882361F08E01045F1F4FF3
:100E50007E010894E11CF11CA4E0DA2ED0CF80E0E2
:100E600001C080EC90E19093F1008093F1008091BB
:100E7000E8008E778093E8002F960FB6F894DEBFD7
:100E80000FBECDBFDF91CF911F910F91FF90EF90DB
:100E9000DF9008951F920F920FB60F9211248F9337
:100EA000199908C08091A30187FF02C02A9A19C02E
:100EB0002A9817C08091A301880F8093A301809185
:100EC000A20181508093A201882321F41092810015
:100ED00082E086BB1B9B05C08091A301816080934B
:100EE000A301199A8F910F900FBE0F901F90189524
:100EF0003E9A10926F00109285001092840081E05B
:100F000090E0909389008093880080E48093800033
:100F100089E080938100089580916701882349F0DA
:100F200084B1897F84B985B1867F85B91CBC1DBC1D
:100F3000089584B1897F84B985B1867F85B9D8CF7A
:100F400092E090936F00109285001092840090E0E0
:100F5000880F991F85559F4FFC012591349130933F
:100F600089002093880010928000109281000895DB
:100F700088E95DDB8730D8F491E090936701E82F32
:100F8000F0E0EE54FF4FE491E061209A289A84B19A
:100F9000866084B923982B9A8DB5E6FF02C08160E4
:100FA00001C08E7F8DBD2098E064ECBD0895109245
:100FB000670194B1966094B995B1996095B9C0CF25
:100FC0008093A30188E08093A2018091A30187FF11
:100FD00002C02A9A01C02A981092850010928400BB
:100FE0008AE0809381008091A201882319F08AB55C
:100FF0008823C9F7109281008091A30108959091F0
:101000006701992329F08EBD0DB407FEFDCF089529
:10101000D7CF882339F0249A8EE909DB882319F485
:101020002C9A089524982C98089580EFE8DF80E0AA
:10103000E6DF80E0E4DF80916701882331F01EBCA9
:101040000DB407FEFDCF8EB502C080E0B9DF80FF92
:1010500003C08AB5882349F78AB5882311F080E058
:10106000089581E808958DE4CADF80E0C8DF8091AB
:10107000A801C5DF80E0C3CF0F931F93CF93DF9309
:10108000EB01142FE82FF0E0EE77E830F10589F15D
:10109000E930F1053CF4E230F10569F0E430F105A6
:1010A00051F50CC0E032F10549F0E034F10509F1E9
:1010B000E031F10501F5822FE8DD1DC0802F9FDFB3
:1010C0008D2F9DDF8C2F9BDF80916701882331F06E
:1010D0001EBC0DB407FEFDCF8EB502C080E070DFF0
:1010E000811719F48AB5882349F78AB5882329F02E
:1010F00002C09BDF03C080E001C080E894E69ABD97
:10110000DF91CF911F910F9108959B01692F782F47
:10111000832F922F0895AF92BF92CF92DF92EF92DA
:10112000FF920F931F93CF93DF93CDB7DEB7C850D5
:10113000D1400FB6F894DEBF0FBECDBFCE010196F1
:1011400068E070E040E050E094D66B817C818D8156
:101150009E81DBDFDC01CB018B839C83AD83BE836F
:101160007F8168856F837887CE01099640E050E0E3
:1011700080D68F81988509968F739070009739F487
:101180008091E8008B778093E8000E94471180915E
:10119000E8008B778093E80082E08093E9008091FB
:1011A000EC0081608093EC008091A401882379F5A4
:1011B00029812150EB80FC800D811E812630A0F416
:1011C00030E0F901E858FE4F4081F901E258FE4F46
:1011D0008081F901EC57FE4F608126573E4FF9019F
:1011E0009081992371F003C066E283E24EE2AF8002
:1011F000B8842A8199E0C92ED12CCC0EDD1E04D4EE
:101200000EC0842FB801A7012985DAD308C04F8109
:1012100058858B819C81BE01675F7F4F87D588236E
:1012200011F080E001C083E090E59093F10094E03C
:101230009093F1008093F1008091E8008E77809385
:10124000E800C85FDE4F0FB6F894DEBF0FBECDBF1B
:10125000DF91CF911F910F91FF90EF90DF90CF9092
:10126000BF90AF900895CF93DF93CDB7DEB7C7504F
:10127000D1400FB6F894DEBF0FBECDBFCE010196B0
:1012800067E070E040E050E0F4D56A817B818C81BA
:101290009D813BDFDC01CB018A839B83AC83BD83D3
:1012A0008E819F819E838F838091E8008B778093CE
:1012B000E80082E08093E9008091EC0081608093F7
:1012C000EC008091A4012E813F81882349F46A813A
:1012D0007B818C819D81AE01485F5F4F37D307C012
:1012E0008A819B81BE01685F7F4FA901F3D4882367
:1012F00011F080E001C083E090E59093F10095E06B
:101300009093F1008093F100882339F46E817F81FE
:10131000CE01089640E050E05CD58091E8008E77E1
:101320008093E800C95FDE4F0FB6F894DEBF0FBEB2
:10133000CDBFDF91CF910895CF93DF930F92CDB7BB
:10134000DEB7CE01019661E070E040E050E091D55B
:101350008091E8008B778093E80082E08093E90039
:101360008091EC0081608093EC0089818093A401DE
:1013700081E58093F1008981813011F080E001C026
:1013800080EC8093F1008091E8008E778093E800F4
:101390000F90DF91CF910895CF93DF93CDB7DEB754
:1013A00029970FB6F894DEBF0FBECDBF8091F10034
:1013B000843009F496C0853048F4823089F1833056
:1013C00008F04AC0813009F029C10AC0863009F40A
:1013D0008CC0863008F487C0873009F01FC1C9C0AF
:1013E0008091E8008B778093E80082E08093E900A9
:1013F0008091EC0081608093EC008091A4018823AF
:1014000011F420D205C0823011F41BD401C080E059
:1014100090E59093F10091E09093F1008927F7C057
:101420009091E8009B779093E8008093E900809189
:10143000EC0081608093EC008091A401882311F47A
:1014400043D201C03CD480E58093F10082E08093D8
:10145000F1001092F100DDC0CE01059665E070E06C
:1014600040E050E006D56E817F81888599854DDE0C
:10147000DC01CB018E839F83A887B9878091E80028
:101480008B778093E80082E08093E9008091EC0004
:1014900081608093EC008091A401ED81882379F430
:1014A000E150E83028F4F0E0E059FE4F808101C0BF
:1014B00080E04E815F816885798517D308C0E1306F
:1014C00011F480E101C084E16E817F8167D48823BB
:1014D00011F080E001C083E090E59093F10093E08B
:1014E00094C019DE9BC0BFDE99C0CE01059661E0B5
:1014F00070E040E050E0BDD48091E8008B778093AD
:10150000E80082E08093E9008091EC0081608093A4
:10151000EC008091A401882391F4ED81E150E23048
:1015200028F4F0E0E057FE4F808101C088E7BE015B
:101530006F5F7F4FD4D1882321F080E003C081E02A
:1015400001C083E090E59093F10096E09093F10064
:101550008093F100882309F05CC089819A81AB8176
:10156000BC81CD01AA27BB278093F10099818A8194
:101570004CC08091F100833031F1843028F4813007
:1015800041F0823081F516C0843011F1853059F573
:1015900024C08091F1009091F1002091F1003091F0
:1015A000F10030936C0120936D0190936E01809354
:1015B0006F0117C08091F1009091F10090936A0142
:1015C00080936B010EC08091F1008093690109C086
:1015D0008091F1008093680104C08091F1008091B6
:1015E000F10080E001C081E09091E8009B7790934A
:1015F000E80092E09093E9009091EC009160909364
:10160000EC0090E59093F10097E09093F1008093C7
:10161000F1008091E8008E778093E80029960FB65C
:10162000F894DEBF0FBECDBFDF91CF9108954D99E5
:10163000FECF4D9BFECF4D99FECF5B9A539A809182
:10164000C9008F7E8093C9008091C9008860809313
:10165000C90081E08093AA0108958091C80086FFA7
:10166000FCCF8091C80080648093C8008091C9003D
:10167000877F8093C9008091C90080618093C900F1
:1016800053985B981092AA0108958091AA0188232B
:1016900009F0E3DF80EC8093C8001092C90010923B
:1016A000CA008AB1877D8AB98BB1837D8BB90895D1
:1016B0008091AA01882309F0D0DF8091C800806C56
:1016C0008093C8001092C9001092CA008AB1877D29
:1016D0008AB98BB1837D8BB924982C980895CF93C8
:1016E000DF930F92CDB7DEB79091AA01992319F439
:1016F00089839DDF89819091C80095FFFCCF9091EF
:10170000C80090649093C8008093CE000F90DF9142
:10171000CF9108958091AA01882309F09EDF8091DE
:10172000C80087FD03C08AB58823C9F78091CE0021
:1017300008958091AA01882309F479DF8CE04D99FE
:10174000FECF4D9BFECF4D99FECF8150C1F708953E
:101750001092AA01249A2C9885E08A95F1F700004E
:101760008AB188628AB952988FE190E09093CD0057
:101770008093CC0088E08093C9008FE68093CA00F4
:10178000D8DFD7CF1092AA018AB188628AB952985D
:101790005B9A85E08A95F1F700008FE190E09093E5
:1017A000CD008093CC0088E08093C9008FE68093C1
:1017B000CA00BFDFBECF1F93CF93DF9300D0CDB75A
:1017C000DEB7182F862F79839A8389DF7981872F57
:1017D00086DF812F84DF9A81892F81DF0F900F9020
:1017E000DF91CF911F91089590E0A0E0B0E040918B
:1017F0006C0150916D0160916E0170916F01842BAD
:10180000952BA62BB72BBC01CD01D5CF80E867DF88
:1018100081DF9AB5992321F081FFF8CF81E0089507
:1018200080E008958BE65BDF8FE0DEDF80E257DF4C
:1018300071DF9AB5992321F087FDF8CF81E00895F3
:1018400080E00895CF92DF92EF92FF920F931F9363
:10185000CF93DF93CDB7DEB728970FB6F894DEBFEE
:101860000FBECDBF8FDF81EC3ADF89E538DF82EC38
:1018700036DF82E034DF80EE32DF8E01075F1F4FFC
:101880007E010894E11CF11C6701F601A2E9B1E0B8
:1018900088E00D9001928150E1F7F80182918F016B
:1018A0001EDF0E151F0589F7B1DF28960FB6F894D5
:1018B000DEBF0FBECDBFDF91CF911F910F91FF9083
:1018C000EF90DF90CF900895A1DF81EC08DF80E0FA
:1018D00006DF81E804DF1EDF8823B9F7D6CE1F9329
:1018E000CF93DF93182FEB01188219821A821B8283
:1018F00099DF882331F18CE4F2DE8AE075DF812FF5
:10190000EEDE8CE4ECDE8BE06FDF81E0E8DE7EDF94
:101910008823B9F087DF8823A1F08BE6E0DE84E03E
:1019200063DF80EADCDE82E0DADE84E2D8DEF2DE4B
:101930008883F0DE8983EEDE8A839AB581E099237D
:1019400009F480E0DF91CF911F910895CF92DF924B
:10195000EF92FF920F931F93CF93DF936B017C0164
:101960008A01E9015FDF882309F18CE4B8DE8AE0AF
:101970003BDF83E4B4DE8BE6B2DEC701B6011BDFDA
:1019800080EAADDE8C2F8150AADE84E2A8DE04C09E
:10199000C1DEF80181938F01209721F08AB521974C
:1019A0008823B1F79AB581E0992309F480E0DF91AB
:1019B000CF911F910F91FF90EF90DF90CF900895FE
:1019C000CF92DF92EF92FF92CF93DF93C82F6A01FD
:1019D0007B01D22F27DF882379F08CE480DE8AE038
:1019E00003DF8C2F7CDE8CE47ADEC701B601E3DEF8
:1019F0008D2F75DE81E001C080E0DF91CF91FF90F7
:101A0000EF90DF90CF9008953F924F925F926F9248
:101A10007F928F929F92AF92BF92CF92DF92EF927E
:101A2000FF920F931F93CF93DF93882E962E342E21
:101A300027013801E601122F20FF10C0F3DE8823B2
:101A400009F440C08CE44BDE8AE0CEDE892D47DE0F
:101A50008CE445DE8BE0C8DE81E041DEA114B104F8
:101A6000E9F0E0DE882371F18CE439DE8AE0BCDE47
:101A7000882D35DE8BE633DEC301B2019CDE80EAC1
:101A80002EDE8A2D81502BDE84E629DE899127DE29
:101A90000894A108B108A114B104C1F711FF10C046
:101AA000C1DE882379F08CE41ADE8AE09DDE832D86
:101AB00016DE8CE414DEC301B2017DDE80E00FDEB1
:101AC00081E001C080E0DF91CF911F910F91FF90E5
:101AD000EF90DF90CF90BF90AF909F908F907F90CE
:101AE0006F905F904F903F900895CF92DF92EF926A
:101AF000FF92CF93C82F6A017B0194DE882309F4FB
:101B000055C08CE4C03429F4EADD8AE06DDE80E45F
:101B100038C0C03309F03CC0E2DD8AE065DE86E310
:101B2000DEDD8CE4DCDD8BE05FDE81E0D8DD7ADEBB
:101B3000882309F43BC08CE4D2DD8AE055DE83E3E0
:101B4000CEDD8BE6CCDDC701B60135DE80EAC7DD30
:101B500080916A018150C3DD84E6C1DDC0E003C02D
:101B600080E0BDDDCF5F2C2F30E080916A01909145
:101B70006B0128173907A0F38CE4B1DD8AE034DE6D
:101B800080E3ADDD8CE4ABDD8BE02EDE81E00BC0CD
:101B9000A6DD8AE029DE8C2FA2DD8CE4A0DDC70162
:101BA000B60109DE80E09BDD31DE01C080E0CF912F
:101BB000FF90EF90DF90CF900895982F9F709069DD
:101BC000282F30E020733070220F331F892F822B93
:101BD00086CD1F93CF93DF930F92CDB7DEB7182F2B
:101BE00088E699837CDD812F7ADD89E678DD99812D
:101BF000892F75DD0F90DF91CF911F91089580E8B7
:101C00006EDD88DD9AB5992321F081FFF8CF81E060
:101C1000089580E0089520916801822F8F7080617F
:101C200030E020733070220F331F822B58DD72DDBD
:101C30009AB5992321F087FDEECF81E0089580E0E9
:101C40000895CF92DF92EF92FF920F931F93CF935D
:101C5000DF93CDB7DEB728970FB6F894DEBF0FBE7F
:101C6000CDBF76DD82EC3BDD82E039DD80EE37DD15
:101C70008E01075F1F4F7E010894E11CF11C670174
:101C8000F601AAE9B1E088E00D9001928150E1F7F8
:101C9000F80182918F0123DD0E151F0589F7AFDF53
:101CA00028960FB6F894DEBF0FBECDBFDF91CF915F
:101CB0001F910F91FF90EF90DF90CF9008959FDFDD
:101CC00080EC0DDD80E00BDD81E809DD23DD88237C
:101CD000B9F7EECCEF92FF920F931F93CF93DF9360
:101CE0007C018B01EA0197DF8823C1F080916901B3
:101CF00064DF80E0F4DCC7016CDF06C084E2EFDC67
:101D000009DDF80181938F01209721F08AB5219791
:101D10008823A1F79AB581E0992309F480E0DF9147
:101D2000CF911F910F91FF90EF900895EF92FF9246
:101D30000F931F93CF93DF937C018B01EA016BDF3D
:101D4000882321F1C0FF06C0F801EC0FFD1F8FEFC3
:101D5000808321968091690130DF8DE1C0DCC7016D
:101D600038DF10C058DF882389F084E6B8DCF8013A
:101D70008081B5DC84E6B3DCF80181810E5F1F4F02
:101D8000AEDC2297209771F781E001C080E0DF91FF
:101D9000CF911F910F91FF90EF9008951F93CF93D4
:101DA000DF93182FEB0137DF882371F080916901F1
:101DB00004DF812F94DCCE0181600BDF80E68FDCB5
:101DC00080E08DDC28DF01C080E0DF91CF911F91A2
:101DD0000895AF92BF92CF92DF92EF92FF921F933E
:101DE000CF93DF93EC017B016A0151D2182F882336
:101DF000A9F5C114D10439F0F60120813181E21A2C
:101E0000F30AC20FD31FAA24BB2423C08091E80089
:101E100085FD16C08091E8008E778093E80059D444
:101E2000C114D10449F0F601808191818A0D9B1D76
:101E30009183808315E012C02AD2882351F00DC00F
:101E400089918093F1000894E108F1080894A11C9D
:101E5000B11CE114F104D1F601C0182F812FDF91DC
:101E6000CF911F91FF90EF90DF90CF90BF90AF90F8
:101E70000895AF92BF92CF92DF92EF92FF921F939D
:101E8000CF93DF93EC017B016A0101D2182F8823E5
:101E9000A9F5C114D10439F0F60120813181E21A8B
:101EA000F30AC20FD31FAA24BB2423C08091E800E9
:101EB00085FD16C08091E8008B778093E80009D4F7
:101EC000C114D10449F0F601808191818A0D9B1DD6
:101ED0009183808315E012C0DAD1882351F00DC0C0
:101EE0008091F10089930894E108F1080894A11CFD
:101EF000B11CE114F104D1F601C0182F812FDF913C
:101F0000CF911F91FF90EF90DF90CF90BF90AF9057
:101F10000895AF92BF92DF92EF92FF920F931F93BB
:101F2000CF93DF93EC017B015A01B1D1D82E8823E6
:101F3000E1F58701015010400C0F1D1FA114B104E1
:101F400039F0F50180819181E81AF90A081B190B13
:101F5000C0E0D0E025C08091E80085FD17C08091E9
:101F6000E8008B778093E800B4D3A114B10451F05A
:101F7000F501808191818C0F9D1F9183808355E0B5
:101F8000D52E13C084D1882359F00EC08091F10062
:101F9000F8018083015010400894E108F10821966F
:101FA000E114F104C1F601C0D82E8D2DDF91CF913F
:101FB0001F910F91FF90EF90DF90BF90AF90089529
:101FC0002091B3013091B4012617370728F4B901E5
:101FD000582F492F20E03EC061157105C9F72091A7
:101FE000E8002E772093E800F3CF8EB3882309F41E
:101FF00046C0853009F43FC08091E80083FD3DC0B4
:102000008091E80082FD31C08091E80080FF22C00D
:102010002091F20030E0E52FF42F2E1B3F0B05C07E
:1020200081918093F10061507040CF01820F931F26
:102030006115710519F08031910590F321E080312F
:10204000910509F020E08091E8008E778093E80008
:102050005E2F4F2F6115710541F6222331F605C021
:102060008EB3882361F0853061F08091E80082FFB3
:10207000F7CF80E0089583E0089581E0089582E03D
:10208000089583E008952091B3013091B40126179B
:10209000370728F4B901582F492F20E03FC06115B8
:1020A0007105C9F72091E8002E772093E800F3CF5F
:1020B0008EB3882309F447C0853009F440C080916D
:1020C000E80083FD3EC08091E80082FD32C080912F
:1020D000E80080FF23C02091F20030E0E52FF42FCC
:1020E0002E1B3F0B06C084918093F1003196615006
:1020F0007040C9018E0F9F1F6115710519F0803165
:10210000910588F321E08031910509F020E080916C
:10211000E8008E778093E8005E2F4F2F61157105E0
:1021200039F6222329F605C08EB3882361F0853065
:1021300061F08091E80082FFF7CF80E0089583E0AE
:10214000089581E0089582E0089583E00895EF9274
:10215000FF920F931F93CF93DF93EB012091B30175
:102160003091B4012617370728F4E901482F392F99
:1021700020E03EC02097D1F72091E8002E772093F1
:10218000E800F4CF8EB3882309F444C0853009F405
:1021900043C08091E80083FD3BC08091E80082FD50
:1021A00031C08091E80080FF23C0E090F200FF245E
:1021B000042F132FE01AF10A07C0C801A5D280939B
:1021C000F1000F5F1F4F2197C8018E0D9F1D2097B3
:1021D00019F08031910588F321E08031910509F0F3
:1021E00020E08091E8008E778093E800402F312F27
:1021F000209741F6222331F605C08EB3882351F093
:10220000853051F08091E80082FFF7CF80E005C073
:1022100081E003C082E001C083E0DF91CF911F9194
:102220000F91FF90EF9008958F708093E900EBEE8F
:10223000F0E0808181608083EDEEF0E010826093B9
:10224000EC0040838091EE00881F8827881F089546
:102250008091AD0187FF11C003C08EB38823B1F018
:102260008091E80082FFF9CF8091E8008B7780931E
:10227000E80008958EB3882349F08091E80080FF3C
:10228000F9CF8091E8008E778093E80008958091DF
:10229000E4009091E50045E601C0C9012091EC0001
:1022A00020FF22C02091E80020FD14C02EB322237D
:1022B00099F0253099F02091EB0025FD11C0209177
:1022C000E4003091E5002817390741F3415029F720
:1022D00084E0089580E0089582E0089583E0089501
:1022E00081E0089580E008952091E80022FFDECF8C
:1022F000F9CF3CD03ED08091D8008F778093D80022
:102300008091D80080688093D8008091D8008F7D1C
:102310008093D80084E089BD86E089BD09B400FEC1
:10232000FDCF1EBA1092AB0180E060E042E17CDF9D
:102330008091E1008E7F8093E1008091E2008160D6
:102340008093E2008091E20088608093E2008091B7
:10235000E0008E7F8093E0000895E3E6F0E0808166
:102360008E7F808381E08093AC01C3CF1092E20026
:1023700008951092E10008951F920F920FB60F92E8
:1023800011242F933F934F935F936F937F938F937A
:102390009F93AF93BF93EF93FF938091E10080FFF2
:1023A00017C08091E20080FF13C08091E2008E7F11
:1023B0008093E2008091E20080618093E20080914E
:1023C000D80080628093D80019BC1EBA0E943A01DE
:1023D0008091E10084FF2DC08091E20084FF29C03C
:1023E00084E089BD86E089BD09B400FEFDCF8091FF
:1023F000D8008F7D8093D8008091E1008F7E8093FC
:10240000E1008091E2008F7E8093E2008091E20003
:1024100081608093E2008091AB01882321F4809158
:10242000E30087FF02C084E001C081E08EBB0E9410
:1024300038018091E10083FF21C08091E20083FF99
:102440001DC08091E100877F8093E10082E08EBB18
:102450001092AB018091E1008E7F8093E10080912A
:10246000E2008E7F8093E2008091E20080618093A1
:10247000E20080E060E042E1D7DE2AD1FF91EF91F7
:10248000BF91AF919F918F917F916F915F914F918C
:102490003F912F910F900FBE0F901F9018951F9393
:1024A000CF93DF9300D00F92CDB7DEB788E0EDEA8F
:1024B000F1E09091F10091938150D9F709D1809189
:1024C000E80083FFF0C08091AD019091AE0195309E
:1024D00009F46CC0963040F4913069F1913070F09D
:1024E000933009F0E0C027C0983009F4AEC09930AD
:1024F00009F4BDC0963009F0D6C07AC0803881F0AA
:10250000823809F0D0C08091B1018F708093E900CA
:102510009091EB0081E095FF80E01092E90001C00E
:1025200080E09091E800977F9093E8008093F1001D
:102530001092F10095C0882319F0823009F0B3C0E1
:102540008F71823009F0AFC08091AF01882341F5CF
:102550002091B1012F7009F4A6C02093E900809169
:10256000EB0080FF1DC08091AE01833021F480918B
:10257000EB00806213C08091EB0080618093EB00E0
:1025800081E090E002C0880F991F2A95E2F78093BE
:10259000EA001092EA008091EB0088608093EB00E3
:1025A0001092E9008091E800877F5DC0882309F0E0
:1025B0007AC01091AF011F778091E3008078812B62
:1025C0008093E3008091E800877F8093E80040DEFD
:1025D0008091E80080FFFCCF8091E30080688093C9
:1025E000E300112311F083E001C082E08EBB5BC0E9
:1025F0008058823008F057C08091AF019091B001AF
:102600006091B101AE014E5F5F4F9E012F5F3F4F62
:102610000E946A01BC01009709F445C08091E8005E
:10262000877F8093E80029818A819B81222311F48E
:102630002ADD05C0213011F48ADD01C0C1DC8091A2
:10264000E8008B778093E8002EC0803861F5809198
:10265000E800877F8093E8008091AB018093F100D0
:102660008091E8008E778093E800F2DD1CC088231B
:10267000D1F49091AF019230B0F48091E800877F5F
:102680008093E8009093AB01E3DD8091AB01882358
:1026900021F48091E30087FF02C084E001C081E063
:1026A0008EBB0E943C018091E80083FF0AC08091AC
:1026B000E800877F8093E8008091EB008062809340
:1026C000EB000F900F900F90DF91CF911F91089525
:1026D0000895CF938EB38823A9F08091E9008F707D
:1026E0009091EC0090FF02C0C0E801C0C0E0C82B90
:1026F0001092E9008091E80083FF01C0D0DECF7026
:10270000C093E900CF910895F999FECF92BD81BDA4
:10271000F89A992780B50895262FF999FECF92BD92
:1027200081BDF89A019700B4021639F01FBA20BD96
:102730000FB6F894FA9AF99A0FBE0895F894FFCF5D
:102740001C03300030003000320030003000300018
:10275000310032003300340035000000000009026F
:102760002000010100C0320904000002FF00000047
:102770000705820240000A0705020240000A41568E
:10278000524953505F4D4B3200800100810100904F
:1027900001009101019201189401219803069E0302
:1027A00001A10100A403000132332000C001000197
:1027B00040206830222A3218242C354C081A232352
:1027C0003323232326263626262601010100000175
:1027D00038391289AB45CDD888FF1289AB45CDD8A1
:0227E00088FF70
:00000001FF
